 jabswitch

 Timestamp is 68fa9027 (Thu Oct 23 20:29:27 2025)

 Preferred load address is 00400000

 Start         Length     Name                   Class
 0001:00000000 000037d1H .text$mn                CODE
 0002:00000000 000001a8H .idata$5                DATA
 0002:000001a8 00000008H .00cfg                  DATA
 0002:000001b0 00000004H .CRT$XCA                DATA
 0002:000001b4 00000004H .CRT$XCAA               DATA
 0002:000001b8 00000004H .CRT$XCZ                DATA
 0002:000001bc 00000004H .CRT$XIA                DATA
 0002:000001c0 00000004H .CRT$XIAA               DATA
 0002:000001c4 00000004H .CRT$XIAC               DATA
 0002:000001c8 00000004H .CRT$XIZ                DATA
 0002:000001cc 00000004H .CRT$XPA                DATA
 0002:000001d0 00000004H .CRT$XPZ                DATA
 0002:000001d4 00000004H .CRT$XTA                DATA
 0002:000001d8 00000008H .CRT$XTZ                DATA
 0002:000001dc 00000000H .gfids$y                DATA
 0002:000001e0 00001120H .rdata                  DATA
 0002:00001300 00000000H .rdata$CastGuardVftablesA DATA
 0002:00001300 00000000H .rdata$CastGuardVftablesC DATA
 0002:00001300 0000012cH .rdata$r                DATA
 0002:0000142c 00000004H .rdata$sxdata           DATA
 0002:00001430 000000a4H .rdata$voltmd           DATA
 0002:000014d4 00000354H .rdata$zzzdbg           DATA
 0002:00001828 00000004H .rtc$IAA                DATA
 0002:0000182c 00000000H .rtc$IMZ                DATA
 0002:0000182c 00000004H .rtc$IZZ                DATA
 0002:00001830 00000004H .rtc$TAA                DATA
 0002:00001834 00000000H .rtc$TMZ                DATA
 0002:00001834 00000004H .rtc$TZZ                DATA
 0002:00001838 000000ecH .xdata$x                DATA
 0002:00001924 00000000H .edata                  DATA
 0002:00001924 00000104H .idata$2                DATA
 0002:00001a28 00000014H .idata$3                DATA
 0002:00001a3c 000001a8H .idata$4                DATA
 0002:00001be4 000007c6H .idata$6                DATA
 0003:00000000 00000048H .data                   DATA
 0003:00000048 00000060H .data$r                 DATA
 0003:000000a8 00000018H .data$rs                DATA
 0003:000000c0 0000038cH .bss                    DATA
 0004:00000000 00000120H .rsrc$01                DATA
 0004:00000120 00000628H .rsrc$02                DATA

  Address         Publics by Value              Rva+Base       Lib:Object

 0000:00000000       ___AbsoluteZero            00000000     <absolute>
 0000:00000000       ___arm64x_extra_rfe_table  00000000     <absolute>
 0000:00000000       ___arm64x_extra_rfe_table_size 00000000     <absolute>
 0000:00000000       ___arm64x_native_entrypoint 00000000     <absolute>
 0000:00000000       ___arm64x_redirection_metadata 00000000     <absolute>
 0000:00000000       ___arm64x_redirection_metadata_count 00000000     <absolute>
 0000:00000000       ___dynamic_value_reloc_table 00000000     <absolute>
 0000:00000000       ___enclave_config          00000000     <absolute>
 0000:00000000       ___guard_check_icall_a64n_fptr 00000000     <absolute>
 0000:00000000       ___guard_eh_cont_count     00000000     <absolute>
 0000:00000000       ___guard_eh_cont_table     00000000     <absolute>
 0000:00000000       ___guard_fids_count        00000000     <absolute>
 0000:00000000       ___guard_fids_table        00000000     <absolute>
 0000:00000000       ___guard_iat_count         00000000     <absolute>
 0000:00000000       ___guard_iat_table         00000000     <absolute>
 0000:00000000       ___guard_longjmp_count     00000000     <absolute>
 0000:00000000       ___guard_longjmp_table     00000000     <absolute>
 0000:00000000       ___hybrid_auxiliary_delayload_iat 00000000     <absolute>
 0000:00000000       ___hybrid_auxiliary_delayload_iat_copy 00000000     <absolute>
 0000:00000000       ___hybrid_auxiliary_iat    00000000     <absolute>
 0000:00000000       ___hybrid_auxiliary_iat_copy 00000000     <absolute>
 0000:00000000       ___hybrid_code_map         00000000     <absolute>
 0000:00000000       ___hybrid_code_map_count   00000000     <absolute>
 0000:00000000       ___hybrid_image_info_bitfield 00000000     <absolute>
 0000:00000000       ___x64_code_ranges_to_entry_points 00000000     <absolute>
 0000:00000000       ___x64_code_ranges_to_entry_points_count 00000000     <absolute>
 0000:00000001       ___safe_se_handler_count   00000001     <absolute>
 0000:00000100       ___guard_flags             00000100     <absolute>
 0000:00000000       ___ImageBase               00400000     <linker-defined>
 0001:00000000       ?isXP@@YA_NXZ              00401000 f   jabswitch.obj
 0001:000000c0       ?enableJAB@@YAXXZ          004010c0 f   jabswitch.obj
 0001:000005a0       ?disableJAB@@YAXXZ         004015a0 f   jabswitch.obj
 0001:00000850       ?modify@@YAH_N@Z           00401850 f   jabswitch.obj
 0001:00000da0       ?printUsage@@YAXXZ         00401da0 f   jabswitch.obj
 0001:00000e80       ?printVersion@@YAXXZ       00401e80 f   jabswitch.obj
 0001:00001110       ?regEnable@@YAHXZ          00402110 f   jabswitch.obj
 0001:000013e0       ?regDeleteValue@@YAHPAUHKEY__@@PB_W@Z 004023e0 f   jabswitch.obj
 0001:00001830       ?regDisable@@YAHXZ         00402830 f   jabswitch.obj
 0001:00001950       _main                      00402950 f   jabswitch.obj
 0001:00001c00       ??$sprintf_s@$0GE@@@YAHAAY0GE@DPBDZZ 00402c00 f i jabswitch.obj
 0001:00001c40       ??$strcat_s@$0BAE@@@YAHAAY0BAE@DPBD@Z 00402c40 f i jabswitch.obj
 0001:00001c70       ??$strcat_s@$0CAA@@@YAHAAY0CAA@DPBD@Z 00402c70 f i jabswitch.obj
 0001:00001ca0       ??$strcat_s@$0GE@@@YAHAAY0GE@DPBD@Z 00402ca0 f i jabswitch.obj
 0001:00001cd0       ??$strcpy_s@$0CAA@@@YAHAAY0CAA@DPBD@Z 00402cd0 f i jabswitch.obj
 0001:00001d00       ??$strcpy_s@$0GE@@@YAHAAY0GE@DPBD@Z 00402d00 f i jabswitch.obj
 0001:00001d30       ?strstr@@YAPADQADQBD@Z     00402d30 f i jabswitch.obj
 0001:00001d50       ?wcsstr@@YAPA_WPA_WPB_W@Z  00402d50 f i jabswitch.obj
 0001:00001d70       ___local_stdio_printf_options 00402d70 f i jabswitch.obj
 0001:00001d80       __vfprintf_l               00402d80 f i jabswitch.obj
 0001:00001dc0       __vsprintf_s_l             00402dc0 f i jabswitch.obj
 0001:00001e40       _fprintf                   00402e40 f i jabswitch.obj
 0001:00001ea0       _printf                    00402ea0 f i jabswitch.obj
 0001:00001f10       _vsprintf_s                00402f10 f i jabswitch.obj
 0001:00001f36       _GetFileVersionInfoSizeW@8 00402f36 f   Version:VERSION.dll
 0001:00001f3c       _GetFileVersionInfoW@16    00402f3c f   Version:VERSION.dll
 0001:00001f42       _VerQueryValueW@16         00402f42 f   Version:VERSION.dll
 0001:00001f48       ??_U@YAPAXI@Z              00402f48 f   MSVCRT:new_array.obj
 0001:00001f51       ___raise_securityfailure   00402f51 f   MSVCRT:gs_report.obj
 0001:00001f79       ___report_gsfailure        00402f79 f   MSVCRT:gs_report.obj
 0001:00002073       ___report_rangecheckfailure 00403073 f   MSVCRT:gs_report.obj
 0001:0000207f       ___report_securityfailure  0040307f f   MSVCRT:gs_report.obj
 0001:0000214e       @_RTC_CheckStackVars@8     0040314e f   MSVCRT:stack.obj
 0001:000021a2       __RTC_CheckEsp             004031a2 f   MSVCRT:stack.obj
 0001:000021c5       @__security_check_cookie@4 004031c5 f   MSVCRT:secchk.obj
 0001:0000241a       _mainCRTStartup            0040341a f   MSVCRT:exe_main.obj
 0001:00002424       ??2@YAPAXI@Z               00403424 f   MSVCRT:new_scalar.obj
 0001:00002454       ?_RTC_Failure@@YAXPAXH@Z   00403454 f   MSVCRT:error.obj
 0001:00002490       ?_RTC_StackFailure@@YAXPAXPBD@Z 00403490 f   MSVCRT:error.obj
 0001:000027ee       ?_RTC_GetErrorFunc@@YAP6AHHPBDH00ZZPBX@Z 004037ee f   MSVCRT:userapi.obj
 0001:000027f4       ?_RTC_GetErrorFuncW@@YAP6AHHPB_WH00ZZPBX@Z 004037f4 f   MSVCRT:userapi.obj
 0001:0000283e       ___scrt_acquire_startup_lock 0040383e f   MSVCRT:utility.obj
 0001:00002870       ___scrt_initialize_crt     00403870 f   MSVCRT:utility.obj
 0001:000028a9       ___scrt_initialize_onexit_tables 004038a9 f   MSVCRT:utility.obj
 0001:00002930       ___scrt_is_nonwritable_in_current_image 00403930 f   MSVCRT:utility.obj
 0001:000029c4       ___scrt_release_startup_lock 004039c4 f   MSVCRT:utility.obj
 0001:000029e1       ___scrt_uninitialize_crt   004039e1 f   MSVCRT:utility.obj
 0001:00002a09       __onexit                   00403a09 f   MSVCRT:utility.obj
 0001:00002a36       _atexit                    00403a36 f   MSVCRT:utility.obj
 0001:00002a98       ___security_init_cookie    00403a98 f   MSVCRT:gs_support.obj
 0001:00002ae3       ___scrt_exe_initialize_mta 00403ae3 f   MSVCRT:utility_desktop.obj
 0001:00002ae3       ___scrt_initialize_winrt   00403ae3 f   MSVCRT:utility_desktop.obj
 0001:00002ae3       ___scrt_stub_for_initialize_mta 00403ae3 f   MSVCRT:utility_desktop.obj
 0001:00002ae3       __get_startup_commit_mode  00403ae3 f   MSVCRT:commit_mode.obj
 0001:00002ae3       __get_startup_new_mode     00403ae3 f   MSVCRT:new_mode.obj
 0001:00002ae3       __get_startup_thread_locale_mode 00403ae3 f   MSVCRT:thread_locale.obj
 0001:00002ae3       __matherr                  00403ae3 f   MSVCRT:matherr.obj
 0001:00002ae6       __get_startup_argv_mode    00403ae6 f   MSVCRT:argv_mode.obj
 0001:00002aea       __get_startup_file_mode    00403aea f   MSVCRT:file_mode.obj
 0001:00002af0       ?__scrt_initialize_type_info@@YAXXZ 00403af0 f   MSVCRT:tncleanup.obj
 0001:00002afc       ___acrt_initialize         00403afc f   MSVCRT:ucrt_stubs.obj
 0001:00002afc       ___acrt_uninitialize       00403afc f   MSVCRT:ucrt_stubs.obj
 0001:00002afc       ___scrt_stub_for_acrt_initialize 00403afc f   MSVCRT:ucrt_stubs.obj
 0001:00002afc       ___scrt_stub_for_acrt_uninitialize 00403afc f   MSVCRT:ucrt_stubs.obj
 0001:00002afc       ___vcrt_initialize         00403afc f   MSVCRT:ucrt_stubs.obj
 0001:00002afc       ___vcrt_uninitialize       00403afc f   MSVCRT:ucrt_stubs.obj
 0001:00002afc       __should_initialize_environment 00403afc f   MSVCRT:env_mode.obj
 0001:00002aff       __initialize_default_precision 00403aff f   MSVCRT:default_precision.obj
 0001:00002b20       @_guard_check_icall_nop@4  00403b20 f   MSVCRT:guard_support.obj
 0001:00002b20       __initialize_denormal_control 00403b20 f   MSVCRT:denormal_control.obj
 0001:00002b20       __initialize_invalid_parameter_handler 00403b20 f   MSVCRT:invalid_parameter_handler.obj
 0001:00002b23       ___local_stdio_scanf_options 00403b23 f i MSVCRT:default_local_stdio_options.obj
 0001:00002b29       ___scrt_initialize_default_local_stdio_options 00403b29 f   MSVCRT:default_local_stdio_options.obj
 0001:00002b46       ___scrt_is_user_matherr_present 00403b46 f   MSVCRT:matherr_detection.obj
 0001:00002b52       ___scrt_get_dyn_tls_init_callback 00403b52 f   MSVCRT:dyn_tls_init.obj
 0001:00002b58       ___scrt_get_dyn_tls_dtor_callback 00403b58 f   MSVCRT:dyn_tls_dtor.obj
 0001:00002b5e       ___scrt_fastfail           00403b5e f   MSVCRT:utility_desktop.obj
 0001:00002c79       ___scrt_initialize_mta     00403c79 f   MSVCRT:utility_desktop.obj
 0001:00002c7e       ___scrt_is_managed_app     00403c7e f   MSVCRT:utility_desktop.obj
 0001:00002cc0       ___scrt_set_unhandled_exception_filter 00403cc0 f   MSVCRT:utility_desktop.obj
 0001:00002ccc       ___scrt_unhandled_exception_filter@4 00403ccc f   MSVCRT:utility_desktop.obj
 0001:00002d22       __crt_debugger_hook        00403d22 f   MSVCRT:utility_desktop.obj
 0001:00002d2a       __RTC_Initialize           00403d2a f   MSVCRT:initsect.obj
 0001:00002d56       __RTC_Terminate            00403d56 f   MSVCRT:initsect.obj
 0001:00002d90       __SEH_prolog4              00403d90 f   MSVCRT:sehprolg4.obj
 0001:00002dd5       __except_handler4          00403dd5 f   MSVCRT:chandler4gs.obj
 0001:00002e04       ??0bad_alloc@std@@QAE@ABV01@@Z 00403e04 f i MSVCRT:throw_bad_alloc.obj
 0001:00002e1f       ??0bad_alloc@std@@QAE@XZ   00403e1f f i MSVCRT:throw_bad_alloc.obj
 0001:00002e37       ??0bad_array_new_length@std@@QAE@ABV01@@Z 00403e37 f i MSVCRT:throw_bad_alloc.obj
 0001:00002e52       ??0bad_array_new_length@std@@QAE@XZ 00403e52 f i MSVCRT:throw_bad_alloc.obj
 0001:00002e6a       ??0exception@std@@QAE@ABV01@@Z 00403e6a f i MSVCRT:throw_bad_alloc.obj
 0001:00002e96       ??1bad_alloc@std@@UAE@XZ   00403e96 f i MSVCRT:throw_bad_alloc.obj
 0001:00002e96       ??1bad_array_new_length@std@@UAE@XZ 00403e96 f i MSVCRT:throw_bad_alloc.obj
 0001:00002ea7       ??_Ebad_alloc@std@@UAEPAXI@Z 00403ea7 f i MSVCRT:throw_bad_alloc.obj
 0001:00002ea7       ??_Ebad_array_new_length@std@@UAEPAXI@Z 00403ea7 f i MSVCRT:throw_bad_alloc.obj
 0001:00002ea7       ??_Eexception@std@@UAEPAXI@Z 00403ea7 f i MSVCRT:throw_bad_alloc.obj
 0001:00002ea7       ??_Gbad_alloc@std@@UAEPAXI@Z 00403ea7 f i MSVCRT:throw_bad_alloc.obj
 0001:00002ea7       ??_Gbad_array_new_length@std@@UAEPAXI@Z 00403ea7 f i MSVCRT:throw_bad_alloc.obj
 0001:00002ea7       ??_Gexception@std@@UAEPAXI@Z 00403ea7 f i MSVCRT:throw_bad_alloc.obj
 0001:00002ed4       ?__scrt_throw_std_bad_alloc@@YAXXZ 00403ed4 f   MSVCRT:throw_bad_alloc.obj
 0001:00002ef1       ?__scrt_throw_std_bad_array_new_length@@YAXXZ 00403ef1 f   MSVCRT:throw_bad_alloc.obj
 0001:00002f0e       ?what@exception@std@@UBEPBDXZ 00403f0e f i MSVCRT:throw_bad_alloc.obj
 0001:00003107       ?_RTC_GetSrcLine@@YAHPAEPA_WKPAH1K@Z 00404107 f   MSVCRT:pdblkup.obj
 0001:00003453       ___isa_available_init      00404453 f   MSVCRT:cpu_disp.obj
 0001:00003627       ___scrt_is_ucrt_dll_in_use 00404627 f   MSVCRT:ucrt_detection.obj
 0001:00003633       ??3@YAXPAXI@Z              00404633 f   MSVCRT:delete_scalar_size.obj
 0001:00003641       ??_Etype_info@@UAEPAXI@Z   00404641 f i MSVCRT:std_type_info_static.obj
 0001:00003641       ??_Gtype_info@@UAEPAXI@Z   00404641 f i MSVCRT:std_type_info_static.obj
 0001:00003664       ??3@YAXPAX@Z               00404664 f   MSVCRT:delete_scalar.obj
 0001:00003669       _memset                    00404669 f   vcruntime:VCRUNTIME140.dll
 0001:0000366f       _strstr                    0040466f f   vcruntime:VCRUNTIME140.dll
 0001:00003675       _wcsstr                    00404675 f   vcruntime:VCRUNTIME140.dll
 0001:0000367b       ___current_exception       0040467b f   vcruntime:VCRUNTIME140.dll
 0001:00003681       ___current_exception_context 00404681 f   vcruntime:VCRUNTIME140.dll
 0001:00003687       __except_handler4_common   00404687 f   vcruntime:VCRUNTIME140.dll
 0001:0000368d       ___std_exception_copy      0040468d f   vcruntime:VCRUNTIME140.dll
 0001:00003693       ___std_exception_destroy   00404693 f   vcruntime:VCRUNTIME140.dll
 0001:00003699       __CxxThrowException@8      00404699 f   vcruntime:VCRUNTIME140.dll
 0001:0000369f       ___vcrt_GetModuleFileNameW 0040469f f   vcruntime:VCRUNTIME140.dll
 0001:000036a5       ___vcrt_LoadLibraryExW     004046a5 f   vcruntime:VCRUNTIME140.dll
 0001:000036ab       _strcpy_s                  004046ab f   ucrt:api-ms-win-crt-string-l1-1-0.dll
 0001:000036b1       _strcat_s                  004046b1 f   ucrt:api-ms-win-crt-string-l1-1-0.dll
 0001:000036b7       _free                      004046b7 f   ucrt:api-ms-win-crt-heap-l1-1-0.dll
 0001:000036bd       _exit                      004046bd f   ucrt:api-ms-win-crt-runtime-l1-1-0.dll
 0001:000036c3       __seh_filter_exe           004046c3 f   ucrt:api-ms-win-crt-runtime-l1-1-0.dll
 0001:000036c9       __set_app_type             004046c9 f   ucrt:api-ms-win-crt-runtime-l1-1-0.dll
 0001:000036cf       ___setusermatherr          004046cf f   ucrt:api-ms-win-crt-math-l1-1-0.dll
 0001:000036d5       __configure_narrow_argv    004046d5 f   ucrt:api-ms-win-crt-runtime-l1-1-0.dll
 0001:000036db       __initialize_narrow_environment 004046db f   ucrt:api-ms-win-crt-runtime-l1-1-0.dll
 0001:000036e1       __get_initial_narrow_environment 004046e1 f   ucrt:api-ms-win-crt-runtime-l1-1-0.dll
 0001:000036e7       __initterm                 004046e7 f   ucrt:api-ms-win-crt-runtime-l1-1-0.dll
 0001:000036ed       __initterm_e               004046ed f   ucrt:api-ms-win-crt-runtime-l1-1-0.dll
 0001:000036f3       __exit                     004046f3 f   ucrt:api-ms-win-crt-runtime-l1-1-0.dll
 0001:000036f9       __set_fmode                004046f9 f   ucrt:api-ms-win-crt-stdio-l1-1-0.dll
 0001:000036ff       ___p___argc                004046ff f   ucrt:api-ms-win-crt-runtime-l1-1-0.dll
 0001:00003705       ___p___argv                00404705 f   ucrt:api-ms-win-crt-runtime-l1-1-0.dll
 0001:0000370b       __cexit                    0040470b f   ucrt:api-ms-win-crt-runtime-l1-1-0.dll
 0001:00003711       __c_exit                   00404711 f   ucrt:api-ms-win-crt-runtime-l1-1-0.dll
 0001:00003717       __register_thread_local_exe_atexit_callback 00404717 f   ucrt:api-ms-win-crt-runtime-l1-1-0.dll
 0001:0000371d       __configthreadlocale       0040471d f   ucrt:api-ms-win-crt-locale-l1-1-0.dll
 0001:00003723       __set_new_mode             00404723 f   ucrt:api-ms-win-crt-heap-l1-1-0.dll
 0001:00003729       ___p__commode              00404729 f   ucrt:api-ms-win-crt-stdio-l1-1-0.dll
 0001:0000372f       __callnewh                 0040472f f   ucrt:api-ms-win-crt-heap-l1-1-0.dll
 0001:00003735       _malloc                    00404735 f   ucrt:api-ms-win-crt-heap-l1-1-0.dll
 0001:0000373b       __initialize_onexit_table  0040473b f   ucrt:api-ms-win-crt-runtime-l1-1-0.dll
 0001:00003741       __register_onexit_function 00404741 f   ucrt:api-ms-win-crt-runtime-l1-1-0.dll
 0001:00003747       __crt_atexit               00404747 f   ucrt:api-ms-win-crt-runtime-l1-1-0.dll
 0001:0000374d       __controlfp_s              0040474d f   ucrt:api-ms-win-crt-runtime-l1-1-0.dll
 0001:00003753       _terminate                 00404753 f   ucrt:api-ms-win-crt-runtime-l1-1-0.dll
 0001:00003759       __filter_x86_sse2_floating_point_exception 00404759 f   MSVCRT:x86_exception_filter.obj
 0001:00003759       __filter_x86_sse2_floating_point_exception_default 00404759 f   MSVCRT:x86_exception_filter.obj
 0002:00000000       __imp__RegOpenKeyExW@20    00405000     Advapi32:ADVAPI32.dll
 0002:00000004       __imp__RegQueryValueExW@24 00405004     Advapi32:ADVAPI32.dll
 0002:00000008       __imp__RegSetValueExW@24   00405008     Advapi32:ADVAPI32.dll
 0002:0000000c       __imp__RegCloseKey@4       0040500c     Advapi32:ADVAPI32.dll
 0002:00000010       \177ADVAPI32_NULL_THUNK_DATA 00405010     Advapi32:ADVAPI32.dll
 0002:00000014       __imp__GetProcAddress@8    00405014     kernel32:KERNEL32.dll
 0002:00000018       __imp__FreeLibrary@4       00405018     kernel32:KERNEL32.dll
 0002:0000001c       __imp__VirtualQuery@12     0040501c     kernel32:KERNEL32.dll
 0002:00000020       __imp__GetProcessHeap@0    00405020     kernel32:KERNEL32.dll
 0002:00000024       __imp__HeapFree@12         00405024     kernel32:KERNEL32.dll
 0002:00000028       __imp__HeapAlloc@12        00405028     kernel32:KERNEL32.dll
 0002:0000002c       __imp__GetCurrentProcessId@0 0040502c     kernel32:KERNEL32.dll
 0002:00000030       __imp__ProcessIdToSessionId@8 00405030     kernel32:KERNEL32.dll
 0002:00000034       __imp__GetVersionExW@4     00405034     kernel32:KERNEL32.dll
 0002:00000038       __imp__GetModuleFileNameW@12 00405038     kernel32:KERNEL32.dll
 0002:0000003c       __imp__UnhandledExceptionFilter@4 0040503c     kernel32:KERNEL32.dll
 0002:00000040       __imp__SetUnhandledExceptionFilter@4 00405040     kernel32:KERNEL32.dll
 0002:00000044       __imp__GetCurrentProcess@0 00405044     kernel32:KERNEL32.dll
 0002:00000048       __imp__TerminateProcess@8  00405048     kernel32:KERNEL32.dll
 0002:0000004c       __imp__IsProcessorFeaturePresent@4 0040504c     kernel32:KERNEL32.dll
 0002:00000050       __imp__IsDebuggerPresent@0 00405050     kernel32:KERNEL32.dll
 0002:00000054       __imp__RaiseException@16   00405054     kernel32:KERNEL32.dll
 0002:00000058       __imp__MultiByteToWideChar@24 00405058     kernel32:KERNEL32.dll
 0002:0000005c       __imp__WideCharToMultiByte@32 0040505c     kernel32:KERNEL32.dll
 0002:00000060       __imp__QueryPerformanceCounter@4 00405060     kernel32:KERNEL32.dll
 0002:00000064       __imp__GetCurrentThreadId@0 00405064     kernel32:KERNEL32.dll
 0002:00000068       __imp__GetSystemTimeAsFileTime@4 00405068     kernel32:KERNEL32.dll
 0002:0000006c       __imp__InitializeSListHead@4 0040506c     kernel32:KERNEL32.dll
 0002:00000070       __imp__GetModuleHandleW@4  00405070     kernel32:KERNEL32.dll
 0002:00000074       __imp__GetLastError@0      00405074     kernel32:KERNEL32.dll
 0002:00000078       \177KERNEL32_NULL_THUNK_DATA 00405078     kernel32:KERNEL32.dll
 0002:0000007c       __imp__wsprintfW           0040507c     User32:USER32.dll
 0002:00000080       \177USER32_NULL_THUNK_DATA 00405080     User32:USER32.dll
 0002:00000084       __imp___CxxThrowException@8 00405084     vcruntime:VCRUNTIME140.dll
 0002:00000088       __imp____std_exception_destroy 00405088     vcruntime:VCRUNTIME140.dll
 0002:0000008c       __imp____vcrt_GetModuleFileNameW 0040508c     vcruntime:VCRUNTIME140.dll
 0002:00000090       __imp____vcrt_LoadLibraryExW 00405090     vcruntime:VCRUNTIME140.dll
 0002:00000094       __imp__memset              00405094     vcruntime:VCRUNTIME140.dll
 0002:00000098       __imp__strstr              00405098     vcruntime:VCRUNTIME140.dll
 0002:0000009c       __imp__wcsstr              0040509c     vcruntime:VCRUNTIME140.dll
 0002:000000a0       __imp____current_exception 004050a0     vcruntime:VCRUNTIME140.dll
 0002:000000a4       __imp____current_exception_context 004050a4     vcruntime:VCRUNTIME140.dll
 0002:000000a8       __imp___except_handler4_common 004050a8     vcruntime:VCRUNTIME140.dll
 0002:000000ac       __imp____std_exception_copy 004050ac     vcruntime:VCRUNTIME140.dll
 0002:000000b0       \177VCRUNTIME140_NULL_THUNK_DATA 004050b0     vcruntime:VCRUNTIME140.dll
 0002:000000b4       __imp__VerQueryValueW@16   004050b4     Version:VERSION.dll
 0002:000000b8       __imp__GetFileVersionInfoW@16 004050b8     Version:VERSION.dll
 0002:000000bc       __imp__GetFileVersionInfoSizeW@8 004050bc     Version:VERSION.dll
 0002:000000c0       \177VERSION_NULL_THUNK_DATA 004050c0     Version:VERSION.dll
 0002:000000c4       __imp___dupenv_s           004050c4     ucrt:api-ms-win-crt-environment-l1-1-0.dll
 0002:000000c8       \177api-ms-win-crt-environment-l1-1-0_NULL_THUNK_DATA 004050c8     ucrt:api-ms-win-crt-environment-l1-1-0.dll
 0002:000000cc       __imp__remove              004050cc     ucrt:api-ms-win-crt-filesystem-l1-1-0.dll
 0002:000000d0       __imp__rename              004050d0     ucrt:api-ms-win-crt-filesystem-l1-1-0.dll
 0002:000000d4       \177api-ms-win-crt-filesystem-l1-1-0_NULL_THUNK_DATA 004050d4     ucrt:api-ms-win-crt-filesystem-l1-1-0.dll
 0002:000000d8       __imp___set_new_mode       004050d8     ucrt:api-ms-win-crt-heap-l1-1-0.dll
 0002:000000dc       __imp___callnewh           004050dc     ucrt:api-ms-win-crt-heap-l1-1-0.dll
 0002:000000e0       __imp__malloc              004050e0     ucrt:api-ms-win-crt-heap-l1-1-0.dll
 0002:000000e4       __imp__free                004050e4     ucrt:api-ms-win-crt-heap-l1-1-0.dll
 0002:000000e8       \177api-ms-win-crt-heap-l1-1-0_NULL_THUNK_DATA 004050e8     ucrt:api-ms-win-crt-heap-l1-1-0.dll
 0002:000000ec       __imp___configthreadlocale 004050ec     ucrt:api-ms-win-crt-locale-l1-1-0.dll
 0002:000000f0       \177api-ms-win-crt-locale-l1-1-0_NULL_THUNK_DATA 004050f0     ucrt:api-ms-win-crt-locale-l1-1-0.dll
 0002:000000f4       __imp____setusermatherr    004050f4     ucrt:api-ms-win-crt-math-l1-1-0.dll
 0002:000000f8       \177api-ms-win-crt-math-l1-1-0_NULL_THUNK_DATA 004050f8     ucrt:api-ms-win-crt-math-l1-1-0.dll
 0002:000000fc       __imp___register_onexit_function 004050fc     ucrt:api-ms-win-crt-runtime-l1-1-0.dll
 0002:00000100       __imp___initialize_onexit_table 00405100     ucrt:api-ms-win-crt-runtime-l1-1-0.dll
 0002:00000104       __imp__terminate           00405104     ucrt:api-ms-win-crt-runtime-l1-1-0.dll
 0002:00000108       __imp___controlfp_s        00405108     ucrt:api-ms-win-crt-runtime-l1-1-0.dll
 0002:0000010c       __imp___errno              0040510c     ucrt:api-ms-win-crt-runtime-l1-1-0.dll
 0002:00000110       __imp__exit                00405110     ucrt:api-ms-win-crt-runtime-l1-1-0.dll
 0002:00000114       __imp__perror              00405114     ucrt:api-ms-win-crt-runtime-l1-1-0.dll
 0002:00000118       __imp___seh_filter_exe     00405118     ucrt:api-ms-win-crt-runtime-l1-1-0.dll
 0002:0000011c       __imp___set_app_type       0040511c     ucrt:api-ms-win-crt-runtime-l1-1-0.dll
 0002:00000120       __imp___cexit              00405120     ucrt:api-ms-win-crt-runtime-l1-1-0.dll
 0002:00000124       __imp___configure_narrow_argv 00405124     ucrt:api-ms-win-crt-runtime-l1-1-0.dll
 0002:00000128       __imp___initialize_narrow_environment 00405128     ucrt:api-ms-win-crt-runtime-l1-1-0.dll
 0002:0000012c       __imp___get_initial_narrow_environment 0040512c     ucrt:api-ms-win-crt-runtime-l1-1-0.dll
 0002:00000130       __imp___initterm           00405130     ucrt:api-ms-win-crt-runtime-l1-1-0.dll
 0002:00000134       __imp___initterm_e         00405134     ucrt:api-ms-win-crt-runtime-l1-1-0.dll
 0002:00000138       __imp___exit               00405138     ucrt:api-ms-win-crt-runtime-l1-1-0.dll
 0002:0000013c       __imp___register_thread_local_exe_atexit_callback 0040513c     ucrt:api-ms-win-crt-runtime-l1-1-0.dll
 0002:00000140       __imp____p___argc          00405140     ucrt:api-ms-win-crt-runtime-l1-1-0.dll
 0002:00000144       __imp____p___argv          00405144     ucrt:api-ms-win-crt-runtime-l1-1-0.dll
 0002:00000148       __imp___c_exit             00405148     ucrt:api-ms-win-crt-runtime-l1-1-0.dll
 0002:0000014c       __imp___crt_atexit         0040514c     ucrt:api-ms-win-crt-runtime-l1-1-0.dll
 0002:00000150       \177api-ms-win-crt-runtime-l1-1-0_NULL_THUNK_DATA 00405150     ucrt:api-ms-win-crt-runtime-l1-1-0.dll
 0002:00000154       __imp____stdio_common_vsprintf_s 00405154     ucrt:api-ms-win-crt-stdio-l1-1-0.dll
 0002:00000158       __imp____p__commode        00405158     ucrt:api-ms-win-crt-stdio-l1-1-0.dll
 0002:0000015c       __imp__fputs               0040515c     ucrt:api-ms-win-crt-stdio-l1-1-0.dll
 0002:00000160       __imp__feof                00405160     ucrt:api-ms-win-crt-stdio-l1-1-0.dll
 0002:00000164       __imp____stdio_common_vfprintf 00405164     ucrt:api-ms-win-crt-stdio-l1-1-0.dll
 0002:00000168       __imp___set_fmode          00405168     ucrt:api-ms-win-crt-stdio-l1-1-0.dll
 0002:0000016c       __imp__fclose              0040516c     ucrt:api-ms-win-crt-stdio-l1-1-0.dll
 0002:00000170       __imp__fopen_s             00405170     ucrt:api-ms-win-crt-stdio-l1-1-0.dll
 0002:00000174       __imp____acrt_iob_func     00405174     ucrt:api-ms-win-crt-stdio-l1-1-0.dll
 0002:00000178       __imp__fgets               00405178     ucrt:api-ms-win-crt-stdio-l1-1-0.dll
 0002:0000017c       \177api-ms-win-crt-stdio-l1-1-0_NULL_THUNK_DATA 0040517c     ucrt:api-ms-win-crt-stdio-l1-1-0.dll
 0002:00000180       __imp__strcat_s            00405180     ucrt:api-ms-win-crt-string-l1-1-0.dll
 0002:00000184       __imp__strtok_s            00405184     ucrt:api-ms-win-crt-string-l1-1-0.dll
 0002:00000188       __imp___stricmp            00405188     ucrt:api-ms-win-crt-string-l1-1-0.dll
 0002:0000018c       __imp__strcpy_s            0040518c     ucrt:api-ms-win-crt-string-l1-1-0.dll
 0002:00000190       __imp___wcslwr_s           00405190     ucrt:api-ms-win-crt-string-l1-1-0.dll
 0002:00000194       __imp__wcscpy_s            00405194     ucrt:api-ms-win-crt-string-l1-1-0.dll
 0002:00000198       __imp__wcslen              00405198     ucrt:api-ms-win-crt-string-l1-1-0.dll
 0002:0000019c       __imp__wcstok_s            0040519c     ucrt:api-ms-win-crt-string-l1-1-0.dll
 0002:000001a0       __imp__wcscat_s            004051a0     ucrt:api-ms-win-crt-string-l1-1-0.dll
 0002:000001a4       \177api-ms-win-crt-string-l1-1-0_NULL_THUNK_DATA 004051a4     ucrt:api-ms-win-crt-string-l1-1-0.dll
 0002:000001a8       ___guard_check_icall_fptr  004051a8     MSVCRT:guard_support.obj
 0002:000001ac       ___castguard_check_failure_os_handled_fptr 004051ac     MSVCRT:guard_support.obj
 0002:000001b0       ___xc_a                    004051b0     MSVCRT:initializers.obj
 0002:000001b8       ___xc_z                    004051b8     MSVCRT:initializers.obj
 0002:000001bc       ___xi_a                    004051bc     MSVCRT:initializers.obj
 0002:000001c8       ___xi_z                    004051c8     MSVCRT:initializers.obj
 0002:000001cc       ___xp_a                    004051cc     MSVCRT:initializers.obj
 0002:000001d0       ___xp_z                    004051d0     MSVCRT:initializers.obj
 0002:000001d4       ___xt_a                    004051d4     MSVCRT:initializers.obj
 0002:000001d8       ___xt_z                    004051d8     MSVCRT:initializers.obj
 0002:00000b78       ??_C@_0NN@JMPELKLB@The?5value?5of?5ESP?5was?5not?5proper@ 00405b78     MSVCRT:error.obj
 0002:00000c58       ??_C@_0BBN@ELNNILBE@A?5cast?5to?5a?5smaller?5data?5type?5h@ 00405c58     MSVCRT:error.obj
 0002:00000d78       ??_C@_0BN@BPOGFMJL@Stack?5memory?5was?5corrupted?$AN?6@ 00405d78     MSVCRT:error.obj
 0002:00000d98       ??_C@_0DG@DAJCDLPN@A?5local?5variable?5was?5used?5befor@ 00405d98     MSVCRT:error.obj
 0002:00000dd0       ??_C@_0CM@JMIDGKLA@Stack?5memory?5around?5_alloca?5was@ 00405dd0     MSVCRT:error.obj
 0002:00000dfc       ??_C@_0BO@CHIONIOI@Unknown?5Runtime?5Check?5Error?$AN?6@ 00405dfc     MSVCRT:error.obj
 0002:00000e20       ??_C@_1GM@CNOOJIHC@?$AAR?$AAu?$AAn?$AAt?$AAi?$AAm?$AAe?$AA?5?$AAC?$AAh?$AAe?$AAc?$AAk?$AA?5?$AAE@ 00405e20     MSVCRT:error.obj
 0002:00000e90       ??_C@_1EA@NFKNIFJP@?$AAR?$AAu?$AAn?$AA?9?$AAT?$AAi?$AAm?$AAe?$AA?5?$AAC?$AAh?$AAe?$AAc?$AAk?$AA?5@ 00405e90     MSVCRT:error.obj
 0002:00000ed0       ??_C@_0BB@PFFGGCJP@Unknown?5Filename@ 00405ed0     MSVCRT:error.obj
 0002:00000ee4       ??_C@_0BE@GNBOBNCK@Unknown?5Module?5Name@ 00405ee4     MSVCRT:error.obj
 0002:00000ef8       ??_C@_0CA@IODNCDPG@Run?9Time?5Check?5Failure?5?$CD?$CFd?5?9?5?$CFs@ 00405ef8     MSVCRT:error.obj
 0002:00000f18       ??_C@_0CG@IAFNJNEE@Stack?5corrupted?5near?5unknown?5va@ 00405f18     MSVCRT:error.obj
 0002:00000f54       ??_C@_0BJ@HEGAHDFO@Stack?5pointer?5corruption@ 00405f54     MSVCRT:userapi.obj
 0002:00000f70       ??_C@_0CK@FEGOIOPB@Cast?5to?5smaller?5type?5causing?5lo@ 00405f70     MSVCRT:userapi.obj
 0002:00000f9c       ??_C@_0BI@CIGMDCBH@Stack?5memory?5corruption@ 00405f9c     MSVCRT:userapi.obj
 0002:00000fb4       ??_C@_0CK@CNLNOEPB@Local?5variable?5used?5before?5init@ 00405fb4     MSVCRT:userapi.obj
 0002:00000fe0       ??_C@_0BP@OGBCLIBO@Stack?5around?5_alloca?5corrupted@ 00405fe0     MSVCRT:userapi.obj
 0002:00001004       ??_7exception@std@@6B@     00406004     MSVCRT:throw_bad_alloc.obj
 0002:0000100c       ??_C@_0BC@EOODALEL@Unknown?5exception@ 0040600c     MSVCRT:throw_bad_alloc.obj
 0002:00001024       ??_7bad_alloc@std@@6B@     00406024     MSVCRT:throw_bad_alloc.obj
 0002:0000102c       ??_C@_0P@GHFPNOJB@bad?5allocation@ 0040602c     MSVCRT:throw_bad_alloc.obj
 0002:00001040       ??_7bad_array_new_length@std@@6B@ 00406040     MSVCRT:throw_bad_alloc.obj
 0002:00001048       ??_C@_0BF@KINCDENJ@bad?5array?5new?5length@ 00406048     MSVCRT:throw_bad_alloc.obj
 0002:00001088       ??_C@_1EI@MLPKHBGE@?$AAa?$AAp?$AAi?$AA?9?$AAm?$AAs?$AA?9?$AAw?$AAi?$AAn?$AA?9?$AAc?$AAo?$AAr?$AAe@ 00406088     MSVCRT:pdblkup.obj
 0002:000010d0       ??_C@_1BK@JHLNAEJL@?$AAa?$AAd?$AAv?$AAa?$AAp?$AAi?$AA3?$AA2?$AA?4?$AAd?$AAl?$AAl@ 004060d0     MSVCRT:pdblkup.obj
 0002:000010ec       ??_C@_0O@COHOBMLB@RegOpenKeyExW@ 004060ec     MSVCRT:pdblkup.obj
 0002:000010fc       ??_C@_0BB@GLNAEDBD@RegQueryValueExW@ 004060fc     MSVCRT:pdblkup.obj
 0002:00001110       ??_C@_0M@HLOHPNFA@RegCloseKey@ 00406110     MSVCRT:pdblkup.obj
 0002:00001120       ??_C@_1HE@EBEAGLFB@?$AAS?$AAO?$AAF?$AAT?$AAW?$AAA?$AAR?$AAE?$AA?2?$AAW?$AAo?$AAw?$AA6?$AA4?$AA3@ 00406120     MSVCRT:pdblkup.obj
 0002:00001194       ??_C@_1BG@EABPBLLF@?$AAP?$AAr?$AAo?$AAd?$AAu?$AAc?$AAt?$AAD?$AAi?$AAr@ 00406194     MSVCRT:pdblkup.obj
 0002:000011ac       ??_C@_0BB@KCIACLNC@PDBOpenValidate5@ 004061ac     MSVCRT:pdblkup.obj
 0002:000011c0       ??_C@_01KDCPPGHE@r@        004061c0     MSVCRT:pdblkup.obj
 0002:000011c8       ??_7type_info@@6B@         004061c8     MSVCRT:std_type_info_static.obj
 0002:000011d0       __load_config_used         004061d0     MSVCRT:loadcfg.obj
 0002:00001300       ??_R4exception@std@@6B@    00406300     MSVCRT:throw_bad_alloc.obj
 0002:00001314       ??_R3exception@std@@8      00406314     MSVCRT:throw_bad_alloc.obj
 0002:00001324       ??_R2exception@std@@8      00406324     MSVCRT:throw_bad_alloc.obj
 0002:0000132c       ??_R1A@?0A@EA@exception@std@@8 0040632c     MSVCRT:throw_bad_alloc.obj
 0002:00001348       ??_R4bad_alloc@std@@6B@    00406348     MSVCRT:throw_bad_alloc.obj
 0002:0000135c       ??_R3bad_alloc@std@@8      0040635c     MSVCRT:throw_bad_alloc.obj
 0002:0000136c       ??_R2bad_alloc@std@@8      0040636c     MSVCRT:throw_bad_alloc.obj
 0002:00001378       ??_R1A@?0A@EA@bad_alloc@std@@8 00406378     MSVCRT:throw_bad_alloc.obj
 0002:00001394       ??_R4bad_array_new_length@std@@6B@ 00406394     MSVCRT:throw_bad_alloc.obj
 0002:000013a8       ??_R3bad_array_new_length@std@@8 004063a8     MSVCRT:throw_bad_alloc.obj
 0002:000013b8       ??_R2bad_array_new_length@std@@8 004063b8     MSVCRT:throw_bad_alloc.obj
 0002:000013c8       ??_R1A@?0A@EA@bad_array_new_length@std@@8 004063c8     MSVCRT:throw_bad_alloc.obj
 0002:000013e4       ??_R4type_info@@6B@        004063e4     MSVCRT:std_type_info_static.obj
 0002:000013f8       ??_R3type_info@@8          004063f8     MSVCRT:std_type_info_static.obj
 0002:00001408       ??_R2type_info@@8          00406408     MSVCRT:std_type_info_static.obj
 0002:00001410       ??_R1A@?0A@EA@type_info@@8 00406410     MSVCRT:std_type_info_static.obj
 0002:0000142c       ___safe_se_handler_table   0040642c     <linker-defined>
 0002:00001430       ___volatile_metadata       00406430     <linker-defined>
 0002:00001828       ___rtc_iaa                 00406828     MSVCRT:initsect.obj
 0002:0000182c       ___rtc_izz                 0040682c     MSVCRT:initsect.obj
 0002:00001830       ___rtc_taa                 00406830     MSVCRT:initsect.obj
 0002:00001834       ___rtc_tzz                 00406834     MSVCRT:initsect.obj
 0002:00001894       __TI2?AVbad_alloc@std@@    00406894     MSVCRT:throw_bad_alloc.obj
 0002:000018a4       __CTA2?AVbad_alloc@std@@   004068a4     MSVCRT:throw_bad_alloc.obj
 0002:000018b0       __CT??_R0?AVbad_alloc@std@@@8??0bad_alloc@std@@QAE@ABV01@@Z12 004068b0     MSVCRT:throw_bad_alloc.obj
 0002:000018cc       __CT??_R0?AVexception@std@@@8??0exception@std@@QAE@ABV01@@Z12 004068cc     MSVCRT:throw_bad_alloc.obj
 0002:000018e8       __TI3?AVbad_array_new_length@std@@ 004068e8     MSVCRT:throw_bad_alloc.obj
 0002:000018f8       __CTA3?AVbad_array_new_length@std@@ 004068f8     MSVCRT:throw_bad_alloc.obj
 0002:00001908       __CT??_R0?AVbad_array_new_length@std@@@8??0bad_array_new_length@std@@QAE@ABV01@@Z12 00406908     MSVCRT:throw_bad_alloc.obj
 0002:00001924       __IMPORT_DESCRIPTOR_ADVAPI32 00406924     Advapi32:ADVAPI32.dll
 0002:00001938       __IMPORT_DESCRIPTOR_VERSION 00406938     Version:VERSION.dll
 0002:0000194c       __IMPORT_DESCRIPTOR_USER32 0040694c     User32:USER32.dll
 0002:00001960       __IMPORT_DESCRIPTOR_KERNEL32 00406960     kernel32:KERNEL32.dll
 0002:00001974       __IMPORT_DESCRIPTOR_VCRUNTIME140 00406974     vcruntime:VCRUNTIME140.dll
 0002:00001988       __IMPORT_DESCRIPTOR_api-ms-win-crt-stdio-l1-1-0 00406988     ucrt:api-ms-win-crt-stdio-l1-1-0.dll
 0002:0000199c       __IMPORT_DESCRIPTOR_api-ms-win-crt-runtime-l1-1-0 0040699c     ucrt:api-ms-win-crt-runtime-l1-1-0.dll
 0002:000019b0       __IMPORT_DESCRIPTOR_api-ms-win-crt-filesystem-l1-1-0 004069b0     ucrt:api-ms-win-crt-filesystem-l1-1-0.dll
 0002:000019c4       __IMPORT_DESCRIPTOR_api-ms-win-crt-string-l1-1-0 004069c4     ucrt:api-ms-win-crt-string-l1-1-0.dll
 0002:000019d8       __IMPORT_DESCRIPTOR_api-ms-win-crt-heap-l1-1-0 004069d8     ucrt:api-ms-win-crt-heap-l1-1-0.dll
 0002:000019ec       __IMPORT_DESCRIPTOR_api-ms-win-crt-environment-l1-1-0 004069ec     ucrt:api-ms-win-crt-environment-l1-1-0.dll
 0002:00001a00       __IMPORT_DESCRIPTOR_api-ms-win-crt-math-l1-1-0 00406a00     ucrt:api-ms-win-crt-math-l1-1-0.dll
 0002:00001a14       __IMPORT_DESCRIPTOR_api-ms-win-crt-locale-l1-1-0 00406a14     ucrt:api-ms-win-crt-locale-l1-1-0.dll
 0002:00001a28       __NULL_IMPORT_DESCRIPTOR   00406a28     Advapi32:ADVAPI32.dll
 0003:00000010       ___security_cookie_complement 00408010     MSVCRT:gs_cookie.obj
 0003:00000014       ___security_cookie         00408014     MSVCRT:gs_cookie.obj
 0003:00000018       ?_RTC_ErrorLevels@@3PAHA   00408018     MSVCRT:error.obj
 0003:0000002c       ___scrt_native_dllmain_reason 0040802c     MSVCRT:utility.obj
 0003:00000030       ___scrt_default_matherr    00408030     MSVCRT:matherr.obj
 0003:00000040       ___isa_enabled             00408040     MSVCRT:cpu_disp.obj
 0003:00000044       ___scrt_ucrt_dll_is_in_use 00408044     MSVCRT:ucrt_stubs.obj
 0003:00000048       ??_R0?AVbad_alloc@std@@@8  00408048     MSVCRT:throw_bad_alloc.obj
 0003:00000064       ??_R0?AVexception@std@@@8  00408064     MSVCRT:throw_bad_alloc.obj
 0003:00000080       ??_R0?AVbad_array_new_length@std@@@8 00408080     MSVCRT:throw_bad_alloc.obj
 0003:000000a8       ??_R0?AVtype_info@@@8      004080a8     MSVCRT:std_type_info_static.obj
 0003:000000c0       ?origFile@@3PAU_iobuf@@A   004080c0     jabswitch.obj
 0003:000000c4       ?tempFile@@3PAU_iobuf@@A   004080c4     jabswitch.obj
 0003:000000c8       ?_OptionsStorage@?1??__local_stdio_printf_options@@9@4_KA 004080c8     jabswitch.obj
 0003:000003fc       ___scrt_current_native_startup_state 004083fc     MSVCRT:utility.obj
 0003:00000400       ___scrt_native_startup_lock 00408400     MSVCRT:utility.obj
 0003:00000420       ?__type_info_root_node@@3U__type_info_node@@A 00408420     MSVCRT:tncleanup.obj
 0003:00000428       ?_OptionsStorage@?1??__local_stdio_scanf_options@@9@4_KA 00408428     MSVCRT:default_local_stdio_options.obj
 0003:00000430       ___scrt_debugger_hook_flag 00408430     MSVCRT:utility_desktop.obj
 0003:0000043c       ___isa_available           0040843c     MSVCRT:cpu_disp.obj
 0003:00000440       ___favor                   00408440     MSVCRT:cpu_disp.obj
 0003:00000444       ___dyn_tls_dtor_callback   00408444     <common>
 0003:00000448       ___dyn_tls_init_callback   00408448     <common>

 entry point at        0001:0000241a

 Static symbols

 0000:ffff5000       .debug$S                   00400000     vcruntime:VCRUNTIME140.dll
 0000:ffff5000       .debug$S                   00400000     vcruntime:VCRUNTIME140.dll
 0000:ffff5000       .debug$S                   00400000     vcruntime:VCRUNTIME140.dll
 0000:ffff5000       .debug$S                   00400000     vcruntime:VCRUNTIME140.dll
 0000:ffff5000       .debug$S                   00400000     vcruntime:VCRUNTIME140.dll
 0000:ffff5000       .debug$S                   00400000     vcruntime:VCRUNTIME140.dll
 0000:ffff5000       .debug$S                   00400000     vcruntime:VCRUNTIME140.dll
 0000:ffff5000       .debug$S                   00400000     vcruntime:VCRUNTIME140.dll
 0000:ffff5000       .debug$S                   00400000     vcruntime:VCRUNTIME140.dll
 0000:ffff5000       .debug$S                   00400000     vcruntime:VCRUNTIME140.dll
 0000:ffff5000       .debug$S                   00400000     vcruntime:VCRUNTIME140.dll
 0000:ffff5000       .debug$S                   00400000     vcruntime:VCRUNTIME140.dll
 0000:ffff5000       .debug$S                   00400000     ucrt:api-ms-win-crt-environment-l1-1-0.dll
 0000:ffff5000       .debug$S                   00400000     ucrt:api-ms-win-crt-filesystem-l1-1-0.dll
 0000:ffff5000       .debug$S                   00400000     ucrt:api-ms-win-crt-filesystem-l1-1-0.dll
 0000:ffff5000       .debug$S                   00400000     ucrt:api-ms-win-crt-heap-l1-1-0.dll
 0000:ffff5000       .debug$S                   00400000     ucrt:api-ms-win-crt-heap-l1-1-0.dll
 0000:ffff5000       .debug$S                   00400000     ucrt:api-ms-win-crt-heap-l1-1-0.dll
 0000:ffff5000       .debug$S                   00400000     ucrt:api-ms-win-crt-heap-l1-1-0.dll
 0000:ffff5000       .debug$S                   00400000     ucrt:api-ms-win-crt-locale-l1-1-0.dll
 0000:ffff5000       .debug$S                   00400000     ucrt:api-ms-win-crt-math-l1-1-0.dll
 0000:ffff5000       .debug$S                   00400000     ucrt:api-ms-win-crt-runtime-l1-1-0.dll
 0000:ffff5000       .debug$S                   00400000     ucrt:api-ms-win-crt-runtime-l1-1-0.dll
 0000:ffff5000       .debug$S                   00400000     ucrt:api-ms-win-crt-runtime-l1-1-0.dll
 0000:ffff5000       .debug$S                   00400000     ucrt:api-ms-win-crt-runtime-l1-1-0.dll
 0000:ffff5000       .debug$S                   00400000     ucrt:api-ms-win-crt-runtime-l1-1-0.dll
 0000:ffff5000       .debug$S                   00400000     ucrt:api-ms-win-crt-runtime-l1-1-0.dll
 0000:ffff5000       .debug$S                   00400000     ucrt:api-ms-win-crt-runtime-l1-1-0.dll
 0000:ffff5000       .debug$S                   00400000     ucrt:api-ms-win-crt-runtime-l1-1-0.dll
 0000:ffff5000       .debug$S                   00400000     ucrt:api-ms-win-crt-runtime-l1-1-0.dll
 0000:ffff5000       .debug$S                   00400000     ucrt:api-ms-win-crt-runtime-l1-1-0.dll
 0000:ffff5000       .debug$S                   00400000     ucrt:api-ms-win-crt-runtime-l1-1-0.dll
 0000:ffff5000       .debug$S                   00400000     ucrt:api-ms-win-crt-runtime-l1-1-0.dll
 0000:ffff5000       .debug$S                   00400000     ucrt:api-ms-win-crt-runtime-l1-1-0.dll
 0000:ffff5000       .debug$S                   00400000     ucrt:api-ms-win-crt-runtime-l1-1-0.dll
 0000:ffff5000       .debug$S                   00400000     ucrt:api-ms-win-crt-runtime-l1-1-0.dll
 0000:ffff5000       .debug$S                   00400000     ucrt:api-ms-win-crt-runtime-l1-1-0.dll
 0000:ffff5000       .debug$S                   00400000     ucrt:api-ms-win-crt-runtime-l1-1-0.dll
 0000:ffff5000       .debug$S                   00400000     ucrt:api-ms-win-crt-runtime-l1-1-0.dll
 0000:ffff5000       .debug$S                   00400000     ucrt:api-ms-win-crt-runtime-l1-1-0.dll
 0000:ffff5000       .debug$S                   00400000     ucrt:api-ms-win-crt-runtime-l1-1-0.dll
 0000:ffff5000       .debug$S                   00400000     ucrt:api-ms-win-crt-runtime-l1-1-0.dll
 0000:ffff5000       .debug$S                   00400000     ucrt:api-ms-win-crt-runtime-l1-1-0.dll
 0000:ffff5000       .debug$S                   00400000     ucrt:api-ms-win-crt-runtime-l1-1-0.dll
 0000:ffff5000       .debug$S                   00400000     ucrt:api-ms-win-crt-runtime-l1-1-0.dll
 0000:ffff5000       .debug$S                   00400000     ucrt:api-ms-win-crt-stdio-l1-1-0.dll
 0000:ffff5000       .debug$S                   00400000     ucrt:api-ms-win-crt-stdio-l1-1-0.dll
 0000:ffff5000       .debug$S                   00400000     ucrt:api-ms-win-crt-stdio-l1-1-0.dll
 0000:ffff5000       .debug$S                   00400000     ucrt:api-ms-win-crt-stdio-l1-1-0.dll
 0000:ffff5000       .debug$S                   00400000     ucrt:api-ms-win-crt-stdio-l1-1-0.dll
 0000:ffff5000       .debug$S                   00400000     ucrt:api-ms-win-crt-stdio-l1-1-0.dll
 0000:ffff5000       .debug$S                   00400000     ucrt:api-ms-win-crt-stdio-l1-1-0.dll
 0000:ffff5000       .debug$S                   00400000     ucrt:api-ms-win-crt-stdio-l1-1-0.dll
 0000:ffff5000       .debug$S                   00400000     ucrt:api-ms-win-crt-stdio-l1-1-0.dll
 0000:ffff5000       .debug$S                   00400000     ucrt:api-ms-win-crt-stdio-l1-1-0.dll
 0000:ffff5000       .debug$S                   00400000     ucrt:api-ms-win-crt-string-l1-1-0.dll
 0000:ffff5000       .debug$S                   00400000     ucrt:api-ms-win-crt-string-l1-1-0.dll
 0000:ffff5000       .debug$S                   00400000     ucrt:api-ms-win-crt-string-l1-1-0.dll
 0000:ffff5000       .debug$S                   00400000     ucrt:api-ms-win-crt-string-l1-1-0.dll
 0000:ffff5000       .debug$S                   00400000     ucrt:api-ms-win-crt-string-l1-1-0.dll
 0000:ffff5000       .debug$S                   00400000     ucrt:api-ms-win-crt-string-l1-1-0.dll
 0000:ffff5000       .debug$S                   00400000     ucrt:api-ms-win-crt-string-l1-1-0.dll
 0000:ffff5000       .debug$S                   00400000     ucrt:api-ms-win-crt-string-l1-1-0.dll
 0000:ffff5000       .debug$S                   00400000     ucrt:api-ms-win-crt-string-l1-1-0.dll
 0000:ffff5000       .debug$S                   00400000     Advapi32:ADVAPI32.dll
 0000:ffff5000       .debug$S                   00400000     Advapi32:ADVAPI32.dll
 0000:ffff5000       .debug$S                   00400000     Advapi32:ADVAPI32.dll
 0000:ffff5000       .debug$S                   00400000     Advapi32:ADVAPI32.dll
 0000:ffff5000       .debug$S                   00400000     User32:USER32.dll
 0000:ffff5000       .debug$S                   00400000     Version:VERSION.dll
 0000:ffff5000       .debug$S                   00400000     Version:VERSION.dll
 0000:ffff5000       .debug$S                   00400000     Version:VERSION.dll
 0000:ffff5000       .debug$S                   00400000     kernel32:KERNEL32.dll
 0000:ffff5000       .debug$S                   00400000     kernel32:KERNEL32.dll
 0000:ffff5000       .debug$S                   00400000     kernel32:KERNEL32.dll
 0000:ffff5000       .debug$S                   00400000     kernel32:KERNEL32.dll
 0000:ffff5000       .debug$S                   00400000     kernel32:KERNEL32.dll
 0000:ffff5000       .debug$S                   00400000     kernel32:KERNEL32.dll
 0000:ffff5000       .debug$S                   00400000     kernel32:KERNEL32.dll
 0000:ffff5000       .debug$S                   00400000     kernel32:KERNEL32.dll
 0000:ffff5000       .debug$S                   00400000     kernel32:KERNEL32.dll
 0000:ffff5000       .debug$S                   00400000     kernel32:KERNEL32.dll
 0000:ffff5000       .debug$S                   00400000     kernel32:KERNEL32.dll
 0000:ffff5000       .debug$S                   00400000     kernel32:KERNEL32.dll
 0000:ffff5000       .debug$S                   00400000     kernel32:KERNEL32.dll
 0000:ffff5000       .debug$S                   00400000     kernel32:KERNEL32.dll
 0000:ffff5000       .debug$S                   00400000     kernel32:KERNEL32.dll
 0000:ffff5000       .debug$S                   00400000     kernel32:KERNEL32.dll
 0000:ffff5000       .debug$S                   00400000     kernel32:KERNEL32.dll
 0000:ffff5000       .debug$S                   00400000     kernel32:KERNEL32.dll
 0000:ffff5000       .debug$S                   00400000     kernel32:KERNEL32.dll
 0000:ffff5000       .debug$S                   00400000     kernel32:KERNEL32.dll
 0000:ffff5000       .debug$S                   00400000     kernel32:KERNEL32.dll
 0000:ffff5000       .debug$S                   00400000     kernel32:KERNEL32.dll
 0000:ffff5000       .debug$S                   00400000     kernel32:KERNEL32.dll
 0000:ffff5000       .debug$S                   00400000     kernel32:KERNEL32.dll
 0000:ffff5000       .debug$S                   00400000     kernel32:KERNEL32.dll
 0000:ffff5000       .debug$S                   00400000     kernel32:KERNEL32.dll
 0001:000000a4       $LN6                       004010a4     jabswitch.obj
 0001:000000ac       $LN5                       004010ac     jabswitch.obj
 0001:000000b8       $LN4                       004010b8     jabswitch.obj
 0001:0000051c       $LN31                      0040151c     jabswitch.obj
 0001:00000524       $LN30                      00401524     jabswitch.obj
 0001:0000056c       $LN29                      0040156c     jabswitch.obj
 0001:00000574       $LN28                      00401574     jabswitch.obj
 0001:0000057c       $LN27                      0040157c     jabswitch.obj
 0001:00000584       $LN26                      00401584     jabswitch.obj
 0001:0000058c       $LN25                      0040158c     jabswitch.obj
 0001:00000598       $LN24                      00401598     jabswitch.obj
 0001:000007f0       $LN19                      004017f0     jabswitch.obj
 0001:000007f8       $LN18                      004017f8     jabswitch.obj
 0001:00000828       $LN17                      00401828     jabswitch.obj
 0001:00000830       $LN16                      00401830     jabswitch.obj
 0001:00000838       $LN15                      00401838     jabswitch.obj
 0001:00000844       $LN14                      00401844     jabswitch.obj
 0001:00000d0c       $LN29                      00401d0c     jabswitch.obj
 0001:00000d14       $LN28                      00401d14     jabswitch.obj
 0001:00000d68       $LN27                      00401d68     jabswitch.obj
 0001:00000d6c       $LN26                      00401d6c     jabswitch.obj
 0001:00000d77       $LN25                      00401d77     jabswitch.obj
 0001:00000d82       $LN24                      00401d82     jabswitch.obj
 0001:00000d86       $LN23                      00401d86     jabswitch.obj
 0001:00000d92       $LN22                      00401d92     jabswitch.obj
 0001:00000d9b       $LN21                      00401d9b     jabswitch.obj
 0001:0000106c       $LN14                      0040206c     jabswitch.obj
 0001:00001074       $LN13                      00402074     jabswitch.obj
 0001:000010bc       $LN12                      004020bc     jabswitch.obj
 0001:000010c9       $LN11                      004020c9     jabswitch.obj
 0001:000010d7       $LN10                      004020d7     jabswitch.obj
 0001:000010dd       $LN9                       004020dd     jabswitch.obj
 0001:000010ea       $LN8                       004020ea     jabswitch.obj
 0001:000010f1       $LN7                       004020f1     jabswitch.obj
 0001:00001384       $LN16                      00402384     jabswitch.obj
 0001:0000138c       $LN15                      0040238c     jabswitch.obj
 0001:000013bc       $LN14                      004023bc     jabswitch.obj
 0001:000013c7       $LN13                      004023c7     jabswitch.obj
 0001:000013d2       $LN12                      004023d2     jabswitch.obj
 0001:000013db       $LN11                      004023db     jabswitch.obj
 0001:000017a4       $LN23                      004027a4     jabswitch.obj
 0001:000017ac       $LN22                      004027ac     jabswitch.obj
 0001:000017f4       $LN21                      004027f4     jabswitch.obj
 0001:000017fe       $LN20                      004027fe     jabswitch.obj
 0001:0000180b       $LN19                      0040280b     jabswitch.obj
 0001:00001816       $LN18                      00402816     jabswitch.obj
 0001:00001821       $LN17                      00402821     jabswitch.obj
 0001:0000182a       $LN16                      0040282a     jabswitch.obj
 0001:00001910       $LN7                       00402910     jabswitch.obj
 0001:00001918       $LN6                       00402918     jabswitch.obj
 0001:00001930       $LN5                       00402930     jabswitch.obj
 0001:0000193c       $LN4                       0040293c     jabswitch.obj
 0001:000021d3       ?pre_c_initialization@@YAHXZ 004031d3 f   MSVCRT:exe_main.obj
 0001:0000227e       ?post_pgo_initialization@@YAHXZ 0040327e f   MSVCRT:exe_main.obj
 0001:00002286       ?pre_cpp_initialization@@YAXXZ 00403286 f   MSVCRT:exe_main.obj
 0001:00002298       ?__scrt_common_main_seh@@YAHXZ 00403298 f   MSVCRT:exe_main.obj
 0001:00002536       ?failwithmessage@@YAXPAXHHPBD@Z 00403536 f   MSVCRT:error.obj
 0001:0000279d       ?notify_debugger@@YAXABUtagEXCEPTION_VISUALCPP_DEBUG_INFO@@@Z 0040379d f   MSVCRT:error.obj
 0001:000027fa       ?find_pe_section@@YAPAU_IMAGE_SECTION_HEADER@@QAEI@Z 004037fa f   MSVCRT:utility.obj
 0001:00002a4b       ___get_entropy             00403a4b f   MSVCRT:gs_support.obj
 0001:00002d90       $$000000                   00403d90     MSVCRT:sehprolg4.obj
 0001:00002f1b       ?GetPdbDllFromInstallPath@@YAPAUHINSTANCE__@@XZ 00403f1b f   MSVCRT:pdblkup.obj
 0002:000001b4       ?pre_cpp_initializer@@3P6AXXZA 004051b4     MSVCRT:exe_main.obj
 0002:000001c0       ?pre_c_initializer@@3P6AHXZA 004051c0     MSVCRT:exe_main.obj
 0002:000001c4       ?post_pgo_initializer@@3P6AHXZA 004051c4     MSVCRT:exe_main.obj
 0002:000001e0       $SG45816                   004051e0     jabswitch.obj
 0002:00000258       $SG45818                   00405258     jabswitch.obj
 0002:000002e0       $SG45820                   004052e0     jabswitch.obj
 0002:000002fc       $SG45822                   004052fc     jabswitch.obj
 0002:0000032c       $SG45850                   0040532c     jabswitch.obj
 0002:00000330       $SG45851                   00405330     jabswitch.obj
 0002:00000370       $SG45852                   00405370     jabswitch.obj
 0002:00000390       $SG45856                   00405390     jabswitch.obj
 0002:000003d4       $SG45861                   004053d4     jabswitch.obj
 0002:000003ec       $SG45862                   004053ec     jabswitch.obj
 0002:000003f0       $SG45867                   004053f0     jabswitch.obj
 0002:00000410       $SG45872                   00405410     jabswitch.obj
 0002:0000042c       $SG45873                   0040542c     jabswitch.obj
 0002:00000430       $SG45896                   00405430     jabswitch.obj
 0002:00000448       $SG45897                   00405448     jabswitch.obj
 0002:0000044c       $SG45900                   0040544c     jabswitch.obj
 0002:00000450       $SG45903                   00405450     jabswitch.obj
 0002:0000046c       $SG45904                   0040546c     jabswitch.obj
 0002:00000470       $SG45907                   00405470     jabswitch.obj
 0002:00000474       $SG45931                   00405474     jabswitch.obj
 0002:00000480       $SG45933                   00405480     jabswitch.obj
 0002:000004a0       $SG45934                   004054a0     jabswitch.obj
 0002:000004a8       $SG45935                   004054a8     jabswitch.obj
 0002:000004c4       $SG45936                   004054c4     jabswitch.obj
 0002:000004e0       $SG45939                   004054e0     jabswitch.obj
 0002:00000514       $SG45940                   00405514     jabswitch.obj
 0002:00000540       $SG45941                   00405540     jabswitch.obj
 0002:00000544       $SG45946                   00405544     jabswitch.obj
 0002:00000548       $SG45949                   00405548     jabswitch.obj
 0002:00000564       $SG45950                   00405564     jabswitch.obj
 0002:00000570       $SG45951                   00405570     jabswitch.obj
 0002:000005b0       $SG45952                   004055b0     jabswitch.obj
 0002:000005d0       $SG45953                   004055d0     jabswitch.obj
 0002:000005d4       $SG45955                   004055d4     jabswitch.obj
 0002:000005f4       $SG45956                   004055f4     jabswitch.obj
 0002:000005fc       $SG45960                   004055fc     jabswitch.obj
 0002:00000618       $SG45961                   00405618     jabswitch.obj
 0002:00000620       $SG45963                   00405620     jabswitch.obj
 0002:0000063c       $SG45964                   0040563c     jabswitch.obj
 0002:00000644       $SG45967                   00405644     jabswitch.obj
 0002:00000678       $SG45968                   00405678     jabswitch.obj
 0002:00000688       $SG45969                   00405688     jabswitch.obj
 0002:000006c4       $SG45970                   004056c4     jabswitch.obj
 0002:000006d4       $SG45971                   004056d4     jabswitch.obj
 0002:00000708       $SG45972                   00405708     jabswitch.obj
 0002:0000073c       $SG45973                   0040573c     jabswitch.obj
 0002:00000760       $SG45974                   00405760     jabswitch.obj
 0002:00000790       $SG45975                   00405790     jabswitch.obj
 0002:00000798       $SG45976                   00405798     jabswitch.obj
 0002:000007d0       $SG45977                   004057d0     jabswitch.obj
 0002:00000808       $SG45978                   00405808     jabswitch.obj
 0002:00000844       $SG45979                   00405844     jabswitch.obj
 0002:00000880       $SG45980                   00405880     jabswitch.obj
 0002:000008bc       $SG45981                   004058bc     jabswitch.obj
 0002:000008f8       $SG45982                   004058f8     jabswitch.obj
 0002:00000920       $SG46008                   00405920     jabswitch.obj
 0002:00000948       $SG46010                   00405948     jabswitch.obj
 0002:0000096c       $SG46012                   0040596c     jabswitch.obj
 0002:0000098c       $SG46014                   0040598c     jabswitch.obj
 0002:00000990       $SG46015                   00405990     jabswitch.obj
 0002:000009b0       $SG46016                   004059b0     jabswitch.obj
 0002:000009c4       $SG46017                   004059c4     jabswitch.obj
 0002:000009d0       $SG46018                   004059d0     jabswitch.obj
 0002:00000a08       $SG46049                   00405a08     jabswitch.obj
 0002:00000a14       $SG46086                   00405a14     jabswitch.obj
 0002:00000a18       $SG46087                   00405a18     jabswitch.obj
 0002:00000a1c       $SG46091                   00405a1c     jabswitch.obj
 0002:00000a20       $SG46092                   00405a20     jabswitch.obj
 0002:00000a24       $SG46105                   00405a24     jabswitch.obj
 0002:00000a30       $SG46118                   00405a30     jabswitch.obj
 0002:00000a34       $SG46119                   00405a34     jabswitch.obj
 0002:00000a38       $SG46123                   00405a38     jabswitch.obj
 0002:00000a44       $SG46124                   00405a44     jabswitch.obj
 0002:00000a50       $SG46128                   00405a50     jabswitch.obj
 0002:00000a58       $SG46129                   00405a58     jabswitch.obj
 0002:00000a60       $SG46134                   00405a60     jabswitch.obj
 0002:00000a6c       $SG46135                   00405a6c     jabswitch.obj
 0002:00000a78       $SG46143                   00405a78     jabswitch.obj
 0002:00000a90       $SG46144                   00405a90     jabswitch.obj
 0002:00000aac       $SG46146                   00405aac     jabswitch.obj
 0002:00000ab4       $SG46147                   00405ab4     jabswitch.obj
 0002:00000abc       $SG46150                   00405abc     jabswitch.obj
 0002:00000ac8       $SG46151                   00405ac8     jabswitch.obj
 0002:00000ad4       _GS_ExceptionPointers      00405ad4     MSVCRT:gs_report.obj
 0002:00000adc       ?_RTC_ErrorMessages@@3QBQBDB 00405adc     MSVCRT:error.obj
 0002:00000af4       ?_RTC_NoFalsePositives@@3QBHB 00405af4     MSVCRT:error.obj
 0002:00000b0c       ?stack_premsg@@3QBDB       00405b0c     MSVCRT:error.obj
 0002:00000b28       ?stack_postmsg@@3QBDB      00405b28     MSVCRT:error.obj
 0002:00000b3c       ?uninit_premsg@@3QBDB      00405b3c     MSVCRT:error.obj
 0002:00000b4c       ?uninit_postmsg@@3QBDB     00405b4c     MSVCRT:error.obj
 0002:00000f40       ?_RTC_errlist@@3QBQBDB     00405f40     MSVCRT:userapi.obj
 0002:00001060       ?mspdbName@@3QB_WB         00406060     MSVCRT:pdblkup.obj
 0002:00001838       __sehtable$?__scrt_common_main_seh@@YAHXZ 00406838     MSVCRT:exe_main.obj
 0002:00001858       __sehtable$?notify_debugger@@YAXABUtagEXCEPTION_VISUALCPP_DEBUG_INFO@@@Z 00406858     MSVCRT:error.obj
 0002:00001878       __sehtable$___scrt_is_nonwritable_in_current_image 00406878     MSVCRT:utility.obj
 0002:00001c28       .idata$6                   00406c28     Advapi32:ADVAPI32.dll
 0002:00001c78       .idata$6                   00406c78     Version:VERSION.dll
 0002:00001c90       .idata$6                   00406c90     User32:USER32.dll
 0002:00001e9e       .idata$6                   00406e9e     kernel32:KERNEL32.dll
 0002:00001f94       .idata$6                   00406f94     vcruntime:VCRUNTIME140.dll
 0002:00002298       .idata$6                   00407298     ucrt:api-ms-win-crt-stdio-l1-1-0.dll
 0002:000022b8       .idata$6                   004072b8     ucrt:api-ms-win-crt-runtime-l1-1-0.dll
 0002:000022da       .idata$6                   004072da     ucrt:api-ms-win-crt-filesystem-l1-1-0.dll
 0002:00002300       .idata$6                   00407300     ucrt:api-ms-win-crt-string-l1-1-0.dll
 0002:00002322       .idata$6                   00407322     ucrt:api-ms-win-crt-heap-l1-1-0.dll
 0002:00002342       .idata$6                   00407342     ucrt:api-ms-win-crt-environment-l1-1-0.dll
 0002:00002368       .idata$6                   00407368     ucrt:api-ms-win-crt-math-l1-1-0.dll
 0002:00002388       .idata$6                   00407388     ucrt:api-ms-win-crt-locale-l1-1-0.dll
 0003:00000000       ?ACCESSIBILITY_USER_KEY@@3PB_WB 00408000     jabswitch.obj
 0003:00000004       ?ACCESSIBILITY_SYSTEM_KEY@@3PB_WB 00408004     jabswitch.obj
 0003:00000008       ?ACCESSIBILITY_CONFIG@@3PB_WB 00408008     jabswitch.obj
 0003:0000000c       ?STR_ACCESSBRIDGE@@3PB_WB  0040800c     jabswitch.obj
 0003:000000d0       ?isXPFlag@?1??isXP@@YA_NXZ@4_NA 004080d0     jabswitch.obj
 0003:000000d8       _GS_ExceptionRecord        004080d8     MSVCRT:gs_report.obj
 0003:00000128       _GS_ContextRecord          00408128     MSVCRT:gs_report.obj
 0003:000003f4       ?_RTC_ErrorReportFunc@@3P6AHHPBDH00ZZA 004083f4     MSVCRT:userapi.obj
 0003:000003f8       ?_RTC_ErrorReportFuncW@@3P6AHHPB_WH00ZZA 004083f8     MSVCRT:userapi.obj
 0003:00000404       ?is_initialized_as_dll@@3_NA 00408404     MSVCRT:utility.obj
 0003:00000405       ?module_local_atexit_table_initialized@@3_NA 00408405     MSVCRT:utility.obj
 0003:00000408       ?module_local_atexit_table@@3U_onexit_table_t@@A 00408408     MSVCRT:utility.obj
 0003:00000414       ?module_local_at_quick_exit_table@@3U_onexit_table_t@@A 00408414     MSVCRT:utility.obj
 0003:00000434       ?mspdb@@3PAUHINSTANCE__@@A 00408434     MSVCRT:pdblkup.obj
 0003:00000438       ?alreadyTried@?1??GetPdbDll@@YAPAUHINSTANCE__@@XZ@4_NA 00408438     MSVCRT:pdblkup.obj
 0003:00000439       ?PDBOK@?1??_RTC_GetSrcLine@@YAHPAEPA_WKPAH1K@Z@4_NA 00408439     MSVCRT:pdblkup.obj
 0004:00000120       $R000000                   00409120     jabswitch.exe.res
 0004:00000338       $R000218                   00409338     jabswitch.exe.res
 0004:000003c8       $R0002A8                   004093c8     jabswitch.exe.res
